:020000040800F2
:10000000780B0024AD020008891700083316000899
:10001000B902000895030008552000080000000000
:100020000000000000000000000000008D17000824
:1000300021040008000000008B1700083D1800088C
:10004000C7020008C7020008C7020008C70200086C
:10005000C7020008C7020008C7020008C70200085C
:10006000C7020008C7020008C7020008C70200084C
:10007000C7020008C7020008C7020008C70200083C
:10008000C7020008C7020008C7020008C70200082C
:10009000C7020008C7020008C7020008C70200081C
:1000A000C7020008C7020008C7020008C70200080C
:1000B000C7020008C7020008C7020008C7020008FC
:1000C000C7020008C7020008C7020008C7020008EC
:1000D000C702000811200008C7020008C702000874
:1000E000C7020008C702000800000000C70200089D
:1000F000C7020008C7020008C7020008C7020008BC
:10010000C7020008C7020008C7020008C7020008AB
:10011000C7020008C7020008C7020008C70200089B
:10012000C7020008C7020008C7020008C70200088B
:10013000C7020008C7020008C7020008C70200087B
:1001400000000000000000000000000000000000AF
:10015000C7020008C7020008C7020008C70200085B
:10016000C7020008C7020008C7020008C70200084B
:10017000C7020008C7020008C7020008C70200083B
:10018000C7020008C7020008C7020008C70200082B
:10019000C7020008C7020008C7020008C70200081B
:1001A000C7020008C7020008C7020008C70200080B
:1001B000C7020008C7020008C7020008C7020008FB
:1001C000C7020008C7020008C7020008C7020008EB
:1001D000C7020008C7020008C7020008C7020008DB
:1001E000C7020008C7020008C7020008C7020008CB
:1001F000C7020008C7020008C7020008C7020008BB
:10020000C7020008C7020008C7020008C7020008AA
:10021000C7020008C7020008C7020008C70200089A
:10022000C7020008C7020008C7020008000000005B
:10023000C7020008C702000800000000C70200084B
:10024000C7020008C7020008C7020008C70200086A
:10025000C7020008C7020008C7020008C70200085A
:10026000C7020008C7020008C7020008C70200084A
:10027000C7020008C7020008C7020008000000000B
:10028000C702000800000000C702000800000000CC
:1002900000000000C7020008DFF80CD000F068F88A
:1002A00000480047F9200008780B002406488047E2
:1002B00006480047FEE7FEE7FEE7FEE7FEE7FEE74B
:1002C000FEE7FEE7FEE7FEE7411800089902000896
:1002D0002DE9F05F0546002092469B46884606467B
:1002E000814640241BE0284641464746224600F00E
:1002F0002FF853465A46C01A914110D3114618465A
:10030000224600F016F82D1A67EB01084F462246E8
:100310000120002100F00DF817EB00094E41201ECE
:10032000A4F10104DFDC484631462A464346BDE8D5
:10033000F09F202A04DB203A00FA02F100207047E7
:100340009140C2F1200320FA03F319439040704713
:10035000202A04DB203A21FA02F00021704721FA1A
:1003600002F3D040C2F12002914008431946704781
:10037000064C074D06E0E06840F0010394E80700F2
:1003800098471034AC42F6D3FFF78AFFB421000837
:10039000D4210008FEE70000F0B5BFF34F8FBFF394
:1003A0006F8F1D4900200860BFF34F8FBFF36F8F21
:1003B0001A4C216841F400312160BFF34F8FBFF325
:1003C0006F8F164970310860BFF34F8F081F0068A8
:1003D00043F6FF75104E1036C0F34E31C0F3C9031B
:1003E00005EA4112184642EA80773760401EFAD289
:1003F000491EF5D2BFF34F8F206840F48030206053
:10040000BFF34F8FBFF36F8F03484C30016841F04B
:1004100004010160F0BD000050EF00E014ED00E0C9
:100420007047000010B528B190F83510022903D0AC
:1004300080214165012010BD1D4A4FF4956301687C
:100440008C189C4207D8042280F83520086820F0D8
:100450000100086029E00C6824F00E040C600168BB
:100460000A440A6822F001020A60016E0A6822F456
:1004700080720A6090F85C30012202FA03F10D4BA1
:100480001960D0E919134B60C16E31B10B6823F4C8
:1004900080730B60D0E91C134B60002180F834108E
:1004A00080F83520016D01B18847002010BD0000A3
:1004B000F0FFFDBF045402580248016841F00101F9
:1004C00001607047200400582DE9F84F6C4C002261
:1004D0004FF0B04A4FF0010B4FF0030E4FF00F09F1
:1004E0000B680BFA02F73B40BB4270D14D68022DFE
:1004F00001D0122D12D1D50800EB850CDCF820605C
:100500005507ED0E09FA05F826EA0806D1F810801D
:1005100008FA05F848EA0608CCF82080D0F80080F0
:10052000560091F804C00EFA06F50CF0030C28EA08
:1005300005080CFA06FC4CEA080CC0F800C0D1F81B
:1005400004C0BCF1010F08D0BCF1020F05D0BCF112
:10055000110F02D0BCF1120F16D1D0F808C0D1F89B
:100560000C802CEA050C08FA06F848EA0C08C0F8DA
:100570000880D0F804C02CEA070C0F79C7F30017E5
:10058000974047EA0C074760C768AF438D68B5409E
:100590003D43C5604D68ED006BD53A4D2E6846F081
:1005A00002062E602D6822F0030606F1B04605F023
:1005B00002050095D6F808C495072F0F09FA07F52C
:1005C0002CEA050C304DA84202D100252EE050E067
:1005D0002E4DA84201D1012528E02D4DA84201D180
:1005E000022523E02B4DA84201D103251EE02A4D10
:1005F000A84201D1042519E0284DA84201D10525C2
:1006000014E0274DA84201D106250FE0254DA84250
:1006100001D107250AE0244DA84201D1082505E0B3
:10062000224DA84201D1092500E00A25BD4045EA36
:100630000C05C6F8085425684E689D43F60300D59E
:100640001D43256065684E689D43B60300D51D4374
:100650006560DAF8005056464F689D43FF0200D5AA
:100660001D43356075684F689D43BF0200D51D432B
:100670007560521C102AFFF433AFBDE8F88F0000FC
:1006800080000058F4440258000002580004025848
:1006900000080258000C02580010025800140258BA
:1006A00000180258001C025800200258002402586A
:1006B0000069084000D0012070470AB101837047EB
:1006C0004183704701488068704700001000002493
:1006D00070B5040011D021684CF6CC40086045F29A
:1006E000555021680860D4E9000141602168A06884
:1006F0008860FFF7E7FF054608E0012070BDFFF7BF
:10070000E1FF401B302801D9032070BD2068C0687C
:100710000028F4D120680269E1688A4201D00161B1
:1007200002E04AF6AA210160002070BD00684AF686
:10073000AA210160002070470248816802781144B4
:100740008160704710000024032010B500F058F8B5
:100750000F2000F007F808B1012010BD00F022F8CA
:10076000002010BD70B50D4D04464FF47A71287805
:10077000B1FBF0F00A490968B1FBF0F000F086FD2A
:1007800048B9102C07D200222146501E00F018F85C
:1007900000206C6070BD012070BD000010000024BE
:1007A000000000247047002809DB012100F01F022F
:1007B00091404009800000F1E020C0F8001170472E
:1007C0000E4BF0B41B68C3F30223C3F10704042CDF
:1007D00000D904241D1D072D01D2002300E0DB1EDB
:1007E000012606FA04F56D1E0D409D409E40761EC2
:1007F000164045EA0601F0BC01F02DBC0CED00E00E
:10080000064A00F0070110684FF6FF03184040EA5F
:100810000120034908431060704700000CED00E020
:100820000000FA0510B500F05BFA084909684FF4BA
:10083000807292FAA2F201F47061B2FA82F2D140AF
:10084000034A515CC8400349086010BD184402586F
:100850008C2100080000002410B500F0FBF90749C6
:100860000968102292FAA2F201F07001B2FA82F243
:10087000D140034A515CC84010BD000020440258DA
:100880008C210008364930B50A68096812F0030265
:10089000344BC1F305311B68334C03F0100324685B
:1008A000DFED320AB7EE001AC4F3CC0414FB03F3F5
:1008B00000EE103A2E4BB8EE400A07D02D4C012A1C
:1008C00001D0022A4AD0B4FBF1F10BE0244C283CC1
:1008D00022689506284A03D52468C4F3C104E2407F
:1008E000B2FBF1F101EE901A1968B8EE612AC1F37A
:1008F000080101EE901A1968F8EE611A40EE201A0C
:1009000031EE810A22EE000AC1F34621491C00EEB5
:10091000901AF8EE600A80EE201AFCEEC10AC0EDD3
:10092000000A1968C1F30641491C00EE901AF8EE5E
:10093000600A80EE201AFCEEC10AC0ED010A1968B7
:10094000C1F30661491C00EE901AF8EE600A80EED1
:10095000201ABCEEC10A80ED020A30BD074ABFE78B
:10096000284402582C4402583C44025800000039E4
:100970003844025800093D000090D00340787D01C2
:10098000364930B50A68096812F00302344BC1F3E6
:1009900005511B68334C03F480732468DFED320A81
:1009A000B7EE001AC4F3CC0414FB03F300EE103AC4
:1009B0002E4BB8EE400A07D02D4C012A01D0022A56
:1009C0004AD0B4FBF1F10BE0244C283C2268950698
:1009D000284A03D52468C4F3C104E240B2FBF1F114
:1009E00001EE901A1968B8EE612AC1F3080101EE10
:1009F000901A1968F8EE611A40EE201A31EE810A59
:100A000022EE000AC1F34621491C00EE901AF8EECE
:100A1000600A80EE201AFCEEC10AC0ED000A1968D7
:100A2000C1F30641491C00EE901AF8EE600A80EE10
:100A3000201AFCEEC10AC0ED010A1968C1F3066173
:100A4000491C00EE901AF8EE600A80EE201ABCEE07
:100A5000C10A80ED020A30BD074ABFE728440258A8
:100A60002C440258444402580000003940440258C3
:100A700000093D000090D00340787D012DE9F0474A
:100A8000DFF8BC9104460E46D9F8000000F00700DC
:100A9000B0420CD2D9F8001021F007013143C9F857
:100AA0000010D9F8000000F00700B0427ED1207895
:100AB000DFF89081800707D5D8F80010E26821F0B0
:100AC0000F011143C8F800102078C00762D0D8F891
:100AD0000010A26821F470611143C8F80010594950
:100AE0006068183902281CD003281DD00968012825
:100AF0001DD04907002960DA524F083F396821F0BC
:100B0000070101433960FFF7DDFD0546606841F2EA
:100B10008831022813D003281ED001288A4627D006
:100B200034E009688903E5E709688901E2E7C90556
:100B3000E0E7FFF7C7FD411B514501D923E08A4695
:100B40003868C0F3C2000228F3D123E0FFF7BAFDF2
:100B5000411B514501D916E08A463868C0F3C200EE
:100B60000328F3D116E0FFF7ADFD411B51450AD82C
:100B70003868C0F3C2000128F5D10BE0FFF7A2FDF1
:100B8000411B514502D90320BDE8F087386810F0B9
:100B9000380FF3D1D9F80010484601F00701B142EF
:100BA0000DD9016821F00701314300E005E0016043
:100BB000006800F00700B04201D00120E4E720788F
:100BC000400707D5D8F80010226921F070011143C1
:100BD000C8F80010207801071B4805D50168626934
:100BE00021F07001114301602178C90605D5016823
:100BF000A26921F4E061114301602078800607D5E5
:100C00001149091D0868E26920F07000104308606E
:100C100000F066F8D8F800104FF4807292FAA2F251
:100C200001F47061B2FA82F2D140084A515CC840C6
:100C3000074908600F20FFF795FD0020A4E700009A
:100C400000200052184402581C4402588C2100080D
:100C50000000002410B5FFF7E5FD084909680122EE
:100C600092FAA2F201F00F01B2FA82F2D140044AE4
:100C7000515CC8400349086010BD00001844025888
:100C80008C2100080400002410B5FFF7E3FF07499A
:100C90000968102292FAA2F201F07001B2FA82F20F
:100CA000D140034A515CC84010BD00001C440258AA
:100CB0008C21000810B5FFF7CDFF074909684FF4F4
:100CC000807292FAA2F201F4E061B2FA82F2D140AB
:100CD000024A515CC84010BD1C4402588C210008D7
:100CE0003548F0B50068364D10F03801334809D06A
:100CF0000411082904D0334E10290BD018290BD029
:100D00002046F0BD29688906FBD52968C1F3C101D9
:100D1000C840F0BD3046F0BD274918310A6809685F
:100D200012F00302284BC1F305111B68274F03F093
:100D300001033F68DFED260AB7EE001AC7F3CC07C0
:100D400017FB03F300EE103A224BB8EE400A06D030
:100D5000012A01D0022A2BD0B4FBF1F008E02A6866
:100D6000920603D52A68C2F3C102D040B0FBF1F06D
:100D700001EE900A1868B8EE612AC0F3080001EE8F
:100D8000900A1868F8EE611A40EE201A31EE810AD6
:100D900022EE000AC0F34620401C00EE900AF8EE56
:100DA000600A80EE201ABCEEC10A10EE100AF0BDF7
:100DB000B6FBF1F0DCE70000104402580090D003CD
:100DC0000044025840787D012C44025834440258B3
:100DD00000000039304402582DE9F05F04460078E5
:100DE000DFF8FC8341F28839DFF8F8A3FE4DC00735
:100DF0004ED0D8F800104046C1F3C20102291AD0E3
:100E00000068C0F3C200032805D1DAF8000000F042
:100E1000030002280FD06068B0F5803F12D010B1F7
:100E2000B0F5A02F19D0286820F4803028602868F9
:100E300020F4802009E02868800329D56068002814
:100E400074D025E0286840F480302860606890B154
:100E5000FFF738FC06464F4609E0286840F480203A
:100E60002860EFE7FFF72EFC801BB8427DD828688A
:100E70008003F7D50CE0FFF725FC06464F4604E05B
:100E8000FFF720FC801BB842F0D828688003F7D415
:100E90002078D64F80075AD5D8F8001040464FF436
:100EA0007C3B11F0380F13D00068C0F3C200032858
:100EB00003D1DAF8000080070AD0E068A8B32968F7
:100EC00021F0190101432960FFF7FCFB06461DE0F4
:100ED0002868400702D5E0680028B1D02868E1689A
:100EE00020F0190008432860FFF7ECFB064604E0F9
:100EF000FFF7E8FB801B0228B8D828684007F7D521
:100F000007E0FFF7DFFB801B0228AFD82868400707
:100F1000F7D538689BFAABF220F47C312069B2FA3D
:100F200082F290400143396011E000E0AEE02868B1
:100F300020F001002860FFF7C5FB064604E0FFF73C
:100F4000C1FB801B022891D828684007F7D420787D
:100F5000C00655D5D8F8001040464FF0F84BC1F305
:100F6000C201012917D0006800E0EDE0C0F3C20023
:100F7000032805D1DAF8000000F0030001280AD0A8
:100F8000E069002828682CD040F080002860FFF736
:100F900099FB064616E02868C00502D5E06980285E
:100FA00074D138689BFAABF220F0F841206AB2FAAB
:100FB00082F290400143396022E0FFF783FB801BFF
:100FC000022899D82868C005F7D538689BFAABF293
:100FD000216AB2FA82F220F0F8409140084338606A
:100FE0000EE020F080002860FFF76CFB064604E06E
:100FF000FFF768FB801B022887D82868C005F7D454
:101000002078000724D5774F60694C37002838686E
:101010000FD040F001003860FFF754FB064604E0B3
:10102000FFF750FB801B02288DD838688007F7D562
:101030000EE020F001003860FFF744FB064604E0B4
:10104000FFF740FB801B02287ED838688007F7D462
:101050002078800623D5A069002828680FD040F4A6
:1010600080502860FFF72EFB064604E0FFF72AFBBE
:10107000801B022868D828688004F7D50FE020F488
:1010800080502860FFF71EFB064605E0D6E0FFF71C
:1010900019FB801B022857D828688004F7D42078D1
:1010A000400744D5524F386840F480703860FFF7ED
:1010B00009FB064604E0FFF705FB801B642843D8C4
:1010C0003868C005F7D5474FA068483701280AD0CF
:1010D00008B1052811D0386820F001003860386860
:1010E00020F0040002E0386840F001003860A06899
:1010F00088B1FFF7E7FA064609E0386840F00400D7
:101100003860F0E7FFF7DEFA811B49451CD83868E4
:101110008007F7D50BE0FFF7D5FA064604E0FFF7A6
:10112000D1FA811B49450FD838688007F7D4606A27
:10113000F0B3D8F80010C1F3C20103297ED0022811
:10114000286820F0807000E079E0286003D0FFF785
:10115000B9FA044687E0FFF7B5FA064604E0FFF760
:10116000B1FA801B02287BD828688001F7D4DAF80E
:10117000001040F2F3329143E26A41EA0211A26A9E
:101180001143CAF8001094F834004FF4FE02218E87
:101190004002491EA0F5007080B2C1F30801084367
:1011A000218F491E02EA0141084394F83C1000E0F7
:1011B0005CE0491E120202EA016108430949083154
:1011C00008600B1D19684FF6F872A06C914392FAF3
:1011D000A2F2B2FA82F2904001431960014809E09C
:1011E000104402582844025800440258044402584B
:1011F00000480258001D0168226C21F00C011143C7
:1012000001600168626C21F0020111430160016814
:1012100041F480310160016841F4003101600168EE
:1012200041F480210160016841F0010101602868FA
:1012300040F080702860FFF745FA01E018E00FE009
:10124000044604E0FFF73EFA001B022808D828688D
:101250008001F7D50AE0FFF735FA001B022802D912
:101260000320BDE8F09F28688001F4D40020F8E74F
:101270000120F6E74FF0E0210428086903D020F0B0
:1012800004000861704740F00400FAE7401EB0F126
:10129000807F10B501D3012010BD4FF0E0246061C4
:1012A0000F21601700F0D7FE0020A0610720206109
:1012B000002010BD7047704790F8791090F87A00C0
:1012C0000843704770B502680446D0691368916896
:1012D00010F00F0F64D0594D03F490760D40354354
:1012E00076D0C50707D0DD0505D501251562E26F6B
:1012F00042F00102E267820708D5CA0706D02568D6
:1013000002222A62E26F42F00402E267420708D535
:10131000CA0706D0256804222A62E26F42F0020260
:10132000E26702070ED503F0200201F080552A4340
:1013300052EAC17206D0256808222A62E26F42F0A2
:101340000802E267E26F002A3AD0800608D503F06F
:10135000200001F08051084302D0204600F05CFBE1
:10136000E06F000703D42068806840062AD5204635
:1013700000F044FB2068816849061ED5816821F091
:1013800040018160606FC0B12D490165606FFFF75A
:1013900049F8002814D0606F016DBDE8704008471F
:1013A000850615D503F0200501F0805635430FD092
:1013B0002046BDE8704000F02FBB2046FFF77BFFC2
:1013C00070BD05E02046FFF776FF0020E067F7E7F5
:1013D000C6024FF020050CD54E020AD5E803106274
:1013E00084F8795084F87A502046BDE87040FFF7C1
:1013F00061BF06060AD503F0800601F400010E4322
:1014000004D02046BDE8704000F096BD41060BD5E3
:10141000590609D51168204621F04001116084F871
:10142000795000F005F9CBE70002C9D55800C7D5BF
:10143000106820F080401060C2E70000010000103A
:10144000E919000810B5040003D094F8790010B130
:1014500007E0012010BD002084F87800204600F04D
:1014600027F8242084F879002068016821F0010120
:101470000160204600F00CFB0128EBD0606B10B13E
:10148000204600F01FFA2068416821F49041416035
:101490002068816821F02A0181602068016841F09C
:1014A000010101602046BDE8104000F06FBA000065
:1014B00010B5006886B01B49884230D11A480168CF
:1014C00041F001010160006800F00100059016483C
:1014D0001030016841F01001016000680121134CD7
:1014E00000F0100005904FF4007000900220CDE94C
:1014F000010103900720694604902046FEF7E4FFAF
:101500004FF48061204600916946FEF7DDFF2520FB
:10151000FFF749F9032225201146FFF751F906B0DC
:1015200010BD000000100140E044025800000258C5
:1015300090F87A30202B4CD1B9B1B2B190F8783014
:10154000012B46D0012380F878304166A0F868204E
:10155000A0F86A20FF228168B1F5805F07D07F2361
:1015600051B1B1F1805F0CD010E0012070470169EA
:1015700021B940F2FF1107E0016909BBA0F86C2016
:1015800004E00169E1B13F21A0F86C100021C167BE
:10159000222280F87A2080F8781001688A6842F068
:1015A00001028A6001680A6892000CD50A6842F458
:1015B00080720A600068816841F08051816006E0B5
:1015C000A0F86C30E2E7086840F4907008600020F2
:1015D000704702207047000030B50068114988420A
:1015E0000CD1114A5088010408D411464FF0000371
:1015F0004404097806D50A2901D0538030BD40F44F
:1016000000400DE00D2909D0084DC0F30D04401C29
:1016100080B2C72829555080EFD830BD40F48040B3
:10162000508030BD001001400C0000242000002438
:101630007047FEE70148FFF779B800006801002411
:10164000064A054B1360C2E9010140F6FF70D06005
:101650001046FFF73DB8000000480058680100241C
:10166000144870B586B0016841F00401016001685A
:1016700001F004010591016841F01001016000686A
:1016800000260325694600F010000590082001247B
:10169000CDE900060848CDE90245FEF715FF2020F8
:1016A0006946CDE900060548CDE90245FEF70CFF85
:1016B00006B070BDE04402580010025800080258FD
:1016C0002DE9F0411C4C01251C4E01281C4F12D065
:1016D000207848B108213046FEF7EAFF68B12021A2
:1016E0003846FEF7E5FF40B108213046FEF7E0FF3F
:1016F000012817D01DE02570ECE70A2000F0D4FC8B
:101700000020207008213046FEF7D2FF28B12021AA
:101710003846FEF7CDFF18B10BE00120BDE8F0819F
:101720000220FBE720213846FEF7C2FF012800D146
:1017300025700020F2E700001C0000240010025871
:10174000000802580E4810B586B0016841F001014A
:101750000160006869460B4C00F001000590022012
:101760000090012001900290032003902046FEF794
:10177000ABFE012220460221FEF79FFF06B010BDFE
:10178000E04402580000025870477047704700005C
:1017900070B5284C9CB0256825F004052560254CC3
:1017A00000260C34256845F440452560256805F47D
:1017B00040451B952568AD04FCD5012400940CAD73
:1017C00003962404019402240994CDE90A41079662
:1017D000082485E80D00CDE910466846FFF7FCFABD
:1017E00088B93F2013900320CDE914064020010161
:1017F000CDE91640CDE9180150201A90022113A816
:10180000FFF73CF910B101201CB070BD0A48016817
:1018100041F0800101600848F430016841F00201A4
:101820000160006800F002001B90FEF745FE0020FA
:10183000EAE700000C48025800440258FEF77CBF5B
:101840001C48016841F4700101601B49086840F0C0
:1018500001000860184A0020103210600A68174B17
:101860001A400A60144A18321060121D1060121DCE
:101870001060114A28321060121D1060121D106095
:10188000121D1060121D1060121D1060121D1060DC
:10189000121D10600A6822F480220A600649603135
:1018A000086001200649C1F80801C00601498039D5
:1018B0000860704788ED00E0004402587FEDF6EACA
:1018C0000080005190F83410C90706D001684A68BA
:1018D000836B22F400321A434A6090F8341089076F
:1018E00006D501684A68C36B22F480321A434A6005
:1018F00090F83410490706D501684A68036C22F451
:1019000080221A434A6090F83410090706D501680E
:101910004A68436C22F400421A434A6090F834103B
:10192000C90606D501688A68836C22F480521A437E
:101930008A6090F83410890606D501688A68C36CFD
:1019400022F400521A438A6090F83410490611D5E7
:1019500001684A68036D22F480121A434A60016DDF
:10196000B1F5801F06D101684A68436D22F4C002B8
:101970001A434A6090F83410090606D501684A688F
:10198000806D22F4002202434A607047F8B50025BA
:101990000446C567FEF796FE0746206800686FF0AC
:1019A0007E46000708D500223B464FF40011204632
:1019B000009600F0FBFA60B92068006840070AD57D
:1019C00000223B464FF480012046009600F0EEFADC
:1019D00008B10320F8BD202084F8790084F87A004B
:1019E000002084F87850F8BD10B5806B0021A0F875
:1019F0006A10A0F86210FFF75EFC10BD01680A686B
:101A000022F490720A6001688A6822F001028A60FA
:101A1000202180F87A10704710B5B0F86C2090F84B
:101A20007A300168222B05D0088B40F0080008832B
:101A3000022010BD898C8368B3F5805F01D10369F2
:101A40006BB11140426E531C43661170B0F86A10BE
:101A5000491E0904090CA0F86A1007D015E0436E6E
:101A600011401980416E891C4166EFE701680A68E0
:101A700022F490720A6001688A6822F001028A608A
:101A8000202180F87A10FFF7A7FD002010BD00008C
:101A90002DE9F04F044600688025FD4B0021D4F865
:101AA00010C087B0A6680F46D4F81C8046EA0C0622
:101AB000D4F814C0A26A4CEA080C46EA0C06324379
:101AC0000668DFF8D0C306EA0C06164306602068F5
:101AD0004268E66822F44052324342602268A069BC
:101AE0009A4201D0266A3043A66AB6F1005F04D15B
:101AF000D4E90B6C46EA0C0630439668DFF898C3CD
:101B000006EA0C06064396602068C26A666A22F0FE
:101B10000F023243C262E14E2068E14AB04210D166
:101B2000126802F03802182A74D005DCCAB3082AF9
:101B30007AD0102A47D179E0202A7BD0282A7CD17C
:101B40007AE0D84EB04209D1126802F00702062AA4
:101B500073D2DFE802F053696B6D6F71D24EB04201
:101B600009D1126802F00702062A66D2DFE802F005
:101B7000465C5E606264CD4EB04209D1126802F0EC
:101B80000702062A59D2DFE802F0394F5153555760
:101B9000C74EB0420BD1126802F00702062A4CD29F
:101BA00000E00EE0DFE802F02A4042444648C14E21
:101BB000B04209D1126802F03802182A38D0BBDCD2
:101BC000B4E74FF0010538E0BB4EB04209D11268CE
:101BD00002F00702062A30D2DFE802F01026282A97
:101BE0002C2EB64EB0420BD1126802F00702062A24
:101BF00023D2DFE802F003191B1D1F2100251CE082
:101C000098421AD1A64A121D126802F00702062A4B
:101C100013D202E00CE007E00CE0DFE802F003057D
:101C200007090B0D022508E0042506E0402504E025
:101C3000082502E0102500E02025DFF864B2A04E60
:101C40009842DFF880A2ABF1540B73D1102D31D044
:101C500006DC022D09D0042D0AD0082D2FD111E069
:101C6000202D29D0402D2AD107E0FEF7F5FD13E005
:101C70006846FEF707FE01980EE003A8FEF780FE17
:101C8000049809E0DBF800105846890610D5006872
:101C9000C0F3C1012AFA01F0002811D06168894619
:101CA00001EB410181420AD8B0EB093F07D808E0B7
:101CB0005046F3E78448F1E74FF40040EEE7012790
:101CC00033E1102D4FF000084ED006DC022D0FD06E
:101CD000042D15D0082D04D12DE0202D4AD0402D03
:101CE00013D00127794AA0F54071914270D9E6E7F7
:101CF000FEF7B2FD626A0023414636F812200DE07D
:101D00006846FEF7BFFD019803E003A8FEF738FE22
:101D100004980023616A36F811201946FEF7D8FAB4
:101D200062680902030241EA10615008181841EB89
:101D3000080115E032E0DBF800105846890609D5A5
:101D400000680023C0F3C1012AFA01F0616A36F885
:101D5000112015E0606A002336F8102050460FE08D
:101D60000023FEF7B5FABDE7606A002336F81020BD
:101D7000554805E0606A002336F810204FF4004013
:101D80000021FEF7A5FA0902020241EA10614FEABA
:101D9000590010184A4641EB0801E1E7E3694FF4A6
:101DA000004293424DD1082D23D005DC8DB1012D89
:101DB00012D0042D06D112E0102D35D0202D3AD0AE
:101DC000402D11D0012721F00F00C1F3420108433B
:101DD0005AE0FEF759FF16E0FEF76CFF13E0684685
:101DE000FEF750FD01980EE003A8FEF7C9FD049828
:101DF00009E0DBF800105846890608D50068C0F3F2
:101E0000C1012AFA01F0616A36F8111010E0606A27
:101E100036F81010BAFBF1F04100606801EB500198
:101E2000B1FBF0F081B2CEE7606A36F810102648B8
:101E3000B0FBF1F0F0E7606A36F81000B2FBF0F0AA
:101E4000EAE7082D4AD00ADC0DB3012D43D0042D5A
:101E50007FF44DAF6846FEF715FD019809E0102D9F
:101E600052D0202D55D0402DF2D103A8FEF788FD89
:101E70000498616A36F81110B0FBF1F1606801EB6B
:101E80005001B1FBF0F080B22168C8604DE01FE066
:101E9000000C0058F369FFCFFFF4FF110010014060
:101EA000544402580044004000480040004C0040A8
:101EB000005000400014014000780040007C0040C9
:101EC0009C2100080090D00300093D00FFFC0F009A
:101ED000FEF7DAFECDE7FEF7EDFECAE7DBF80020FD
:101EE000594692060AD50968C1F3C1022AFA02F1DD
:101EF000626A36F81220B1FBF2F20FE0616A36F83E
:101F00001120BAFBF2F209E0616A36F811200949A2
:101F1000F1E7616A36F81110B2FBF1F2616802EB89
:101F20005102B2FBF1F189B2C16007B03846BDE899
:101F3000F08F000000093D0090F87910212901D0B0
:101F400002207047B0F8621021B18168B1F5805F5E
:101F500013D014E001680A68920004D58A6822F45C
:101F600000028A6003E00A6822F080020A600068CA
:101F7000016841F0400101600CE0016961B1C16D8F
:101F80004A1CC265026809781185B0F86210491EC2
:101F9000A0F8621000207047C16D02680988C1F383
:101FA00008011185C16D891CC165EEE72DE9F0417D
:101FB0001E46174688460446069D1CE0681C1AD03B
:101FC00025B1FEF77FFB801BA84214D92068016869
:101FD00021F4D07101602068816821F001018160E5
:101FE000202084F8790084F87A00002084F87800B2
:101FF0000320BDE8F0812068C16938EA010004D0FF
:102000000020B842DAD00020F3E70120F9E7000011
:1020100070B50D4D00240D48FFF754F902E0641C23
:10202000AC4204D80948FFF747F92028F7D100242B
:1020300002E0641CAC4206D8054901220348FFF7C0
:1020400077FA0028F5D170BDFFFF0100E8000024F9
:102050000C000024FEE70907090E002804DB00F14C
:10206000E02080F80014704700F00F0000F1E0203D
:1020700080F8141D704702E008C8121F08C1002A2A
:10208000FAD170477047002001E001C1121F002AF9
:10209000FBD1704710B504460420FFF7EBF8014868
:1020A000046010BD0800002470B5002405464FF4FC
:1020B0007A7603E0304600F005F8641CAC42F9D3B0
:1020C00070BD000070B54FF0E02500216C69094A31
:1020D000AB6912685043AA699A42FCD002D2A3EBC2
:1020E000020302E0A4EB0206334419441346814282
:1020F000F1D370BD08000024FEF74EF9FEF724FB73
:10210000042302220521A020FFF742FB4FF4C870F0
:10211000FFF7C0FF4FF4E13000F01CF8FFF712FBAF
:10212000FFF79EFA04204FF4FA71FFF789FA084886
:1021300000220221FEF7C1FA0020FFF7C1FA0228AF
:1021400001D1FFF777FA0A20FFF7AEFFF4E70000AE
:10215000000002580B490A4A10B5C1E900200020CE
:102160008860C860086188610C2048610846FFF7F4
:1021700069F9BDE81040044901220248FFF7D8B9C7
:1021800000100140E80000240C00002400000000C2
:10219000010203040102030406070809010002000A
:1021A0000400060008000A000C0010002000400097
:1021B00080000001D421000800000024200000005D
:1021C00076200008F421000820000024580B0000AD
:1021D000862000080090D0030090D003000000008B
:1021E00000000000010000001000000000000000DE
:0421F00001000000EA
:040000050800029954
:00000001FF
